:030000000219FDE5
:03000B000200AA46
:03002B0002015679
:03005B000202E2BC
:030073000202CFB7
:1000800002030406080C10182030406080040608A3
:100090000C10182030406080A0C00003070F1F0D17
:1000A0000D0403060D0502030202C2AFC0D0C0E07A
:1000B000206214E5256009E473E525F4F58AD2622F
:1000C000D0E0D0D0D2AF3285268AC262E526F46075
:1000D00029D0E0D0D0D297D295D293D2AF32D29756
:1000E000D295D293206F0C206509740AD5E0FDE506
:1000F0007B4290D0E0D0D0D2AF32758A00C28DD290
:100100006201F301B9306805206502C29701B93078
:100110006805206502C29501B9306805206502C2F4
:100120009301B9C29630680A2065077408D5E0FDCE
:10013000C29701B9C29430680A2065077408D5E0F7
:10014000FDC29501B9C29230680A2065077408D5CE
:10015000E0FDC29301B9C2AFC2AD53E6EFC0D0C05B
:10016000E0D2D3D2AFC2CEE52A6007207449152A67
:1001700021B77800790020742EE580307E01F430BC
:10018000E50278FF53DACF207E0343DA20307E0386
:1001900043DA10C2D8C271E580307E01F430E50246
:1001A00079FFC3E89970CB306103752A402074034E
:1001B000752A40885CD27020740DE52B6004152BE5
:1001C00021C743DA01C2D820700221DAA85C20617D
:1001D00002C27020740221D888227882B604038576
:1001E000222420CF0AD0E0D0D043E610D2AD32C2D4
:1001F000CF053A7802E52A6005307402152AC3E576
:100200005C94014005755F00411B756000756900D5
:10021000E55F2401F55F5003755FFF7982B7020D3A
:10022000306E1DC3E52294324016854C227982B788
:10023000030E306E0BC3E52294324004798E872280
:10024000C3E5239522600840041523414F0523D8B8
:10025000CA0569E56970021569D56A69756A017828
:1002600008E56B60497805C3E569956B4057C3E5C0
:1002700069956C50087801756A03020289C3E569C3
:10028000956D50057801756A01C3E5629524401E9D
:100290007982B7040241BA206E14852462E56904AC
:1002A0006003856B69756A0175233C0202C5E562CE
:1002B0002850057562FF41BAF562E5620470067563
:1002C00060FF7569FFD0E0D0D043E610D2AD32C2F6
:1002D000AF53E67F7592FA7593FFC260759104D2B1
:1002E000AF32C2AF53E6EFC2ADC0D0C0E0C0F0D273
:1002F000D3D2AFA8FBA9FCC2D8307102614953DA4E
:10030000CF207E0343DA10307E0343DA20D271E53A
:1003100080307E01F420E502612088278928A12E03
:1003200053DACF207E0343DA20307E0343DA10C253
:10033000D8C271307402A11A7800E580307E01F4D1
:1003400030E502A11A885CA10253DACF207E034374
:10035000DA20307E0343DA10C27120610281225319
:10036000DACF207E0343DA10307E0343DA20C2D88E
:10037000D27188578958C3E89555F8E99556F97BA5
:10038000007E087A00C3E8948CE994005005755B00
:10039000008114882178A2E6A8216055C3E894C89A
:1003A000E994005008E4D2E4FB7A0A61EFC3E894D0
:1003B00068E994015008E4D2E3FB7A0F61EFC3E8E7
:1003C00094D0E994025008E4D2E2FB7A1E61EFC3B4
:1003D000E894A0E994055008E4D2E1FB7A3C61EF8F
:1003E000C3E89498E994085008E4D2E0FB7A787E58
:1003F00000C3E89559FCE9955AFD30E70AECF4246E
:1004000001FCEDF43400FD755B00C3EC9AED9E50E9
:1004100003755B018859895A855755855856780266
:10042000A102C3E89527F8E99528F9307C0281E616
:10043000307B0281E6307A0281DF2075028145E956
:10044000FDE8FC8164E9C313F9E813F8307902810F
:10045000DFE9C313F9E813F830780281DFE9C31349
:10046000FDE813FC20612CC3EC941CED94024002C7
:0F047000817BED701EC3EC94C850180529E52957
:10047F0070021529C3E529940A5002A11A755C0070
:10048F00D270A11AE529600215297400207F037824
:10049F0096E624FAFEE43400FFC3EC9EFCED9FFDCC
:1004AF0050067800790081E6C3EC94FFED9400408C
:1004BF000678FF790081E6EC8572F0A4C5F0A2F70B
:1004CF0033F87900400302050278FF790002050234
:1004DF00E9C313F9E813F8307C0EE9600278FFC323
:1004EF00E81338F8E43400F9C3E894FFE9940040C6
:1004FF000278FF885CD270206102A11A741FF45534
:10050F002F4BF52FC274EB7002D274752A403074E2
:10051F0003752A0A306102A12E20740353DAFE20DC
:10052F007403752B20D0F0D0E0D0D0D2AD43E610BD
:10053F0032790102055E790302055E790A02055ED2
:10054F00791E02055E796402055E79C802055E7840
:10055F0017E4D5E0FDD8FAD9F6227A147B78020594
:10056F00857A107B8C0205857A0D7BB40205857A1E
:10057F000B7BC8020585E573D5E001227902E4C241
:10058F0094D5E0FDC295D5E0FDD295D5E0FDD2948E
:10059F00D5E0FDE920E002C29730E002C293E57397
:1005AF00D5E0FDE920E002D29730E002D2937496B5
:1005BF00D5E0FDD9C9EAF8D5E0FDD8FBDBB8C29488
:1005CF0022C37C007D0075F00005F0EA33FAEB33AF
:1005DF00FB50F6EB13FBEA13FAC3E9FFE8FEE89AC8
:1005EF00F8E99BF95004EFF9EEF8B3EC33FCED3377
:1005FF00FDD5F0DFEDF9ECF822E889F08A20D2D4AE
:10060F00F8A9F07B0030F70B7BFFF42401F8E9F435
:10061F003400F9E88520F0A4ADF0F8E98520F0A4C6
:10062F00AFF0FEED2EF974003FFA7C04C3EA13FA23
:10063F00E913F9E813F8DCF48BF030F70AE8F42447
:10064F0001F8E9F43400F9E889F0C2D4F8A9F022EE
:10065F007882B604030206FEC3E55C9419401EE5DA
:10066F002D54067018206E3678057994E7146007BC
:10067F00780A1460027812C3E54198401F306E0962
:10068F008564627569FF756A01852224E4F544F576
:10069F0045F546F547F548C26E0206FED26E7994CF
:1006AF00E7147013E523F43333F913F8E954010415
:1006BF00F9E854FE0206F2E714147014E523F4333C
:1006CF003333F913F8E9540304F9E854FC0206FA3A
:1006DF00E523F433333333F913F8E954070404F9FA
:1006EF00E854F8C39440F8E99400F9884489452206
:1006FF00C3E54113F9E54013F8C3E54498F8E54520
:10070F0099F9500CC3E89480E994FF40160207361C
:10071F00C3E8947FE994005003020736787F79008D
:10072F00020736788079FF8849894A22E5492546AC
:10073F00F8E54A3547F9854A20E4300701F4354892
:10074F00FA30E709C3EA94F04015020774C3EA943C
:10075F000F500302077478FF79FF7A0F020774783E
:10076F000079007AF0C3E5249561500AC3740195AE
:10077F0024500B020792E54A20E70E020792E54A42
:10078F0030E706884689478A482278A5E6FAC3E506
:10079F004933F8E54A33F9D108E930E70BC3E89458
:1007AF0080E994FF4013E1CCC3E8947FE9940050B3
:1007BF0002E1CC787F7900E1CC788079FFE820E7FF
:1007CF0015C3E52398F84009C3E8940140030207D5
:1007DF00F378010207F3E8F424012523F84003021C
:1007EF0007F378FF884B2278A6E6FAA847A94812A4
:1007FF000608E930E70CC3E89401E994FF401602BC
:10080F000828C3E894FFE99400500302082878FFF2
:10081F007900020828780179FFE920E715C3E54B35
:10082F0098F84009C3E89401400302084F78010289
:10083F00084FE8F42401254BF8400302084F78FFD6
:10084F0088242278FF20692879A1E76023E5416099
:10085F001F74FF8541F0848539F0306A0375F00508
:0E086F00A4F8C5F0600278FFC3E8956450025B
:10087D00A864886322C3E5409440E5419401E56393
:10088D005003140193046002F563227883E6F5208A
:10089D00120F1375E89012054075E89030EDFDA824
:1008AD00BDA9BE120FB9756E55756F00C3740013D7
:1008BD00FD7455606613FC74552CFC74003DFDEC05
:1008CD00FAEDFBC3E89AE99B4014E56E2455F56EED
:1008DD00E56F3400F56FEA2CFAEB3DFB80E5AE6E6B
:1008ED00AF6FC3E56F13F9E56E13F8C3E913F9E8BC
:1008FD0013F87A03C3E913F9E813F8DAF7AA201A03
:10090D007009756E00756F000209281AEA6008EE0D
:10091D0028FEEF39FFDAF88E6E8F6F2275E8902280
:10092D007883E6FF30EDF9A8BDA9BE0570C3E5706B
:10093D0094084052757000E9FA79A0E76044EA70B6
:10094D0007E571601B020961C3E895716010E571DF
:10095D005006600C1402096D0460F902096DE57111
:10096D00F571C3946D401B7561C0C394044013753C
:10097D006180C39404400B756140C39404400375BA
:10098D00610075BB0822EFC39401601F7455601B95
:10099D00C3E894FFE994035012C3E8956EE9956F8F
:1009AD005009E561600C15610209BFE561F4600253
:1009BD000561A861C3E524985002A824C3E8956297
:1009CD00400AA862E562F460038562618825882685
:1009DD00E570B4070375BB1022743279A787F0A4B4
:1009ED00C5F0A2F733F8C3E895614002A8618822EB
:1009FD008824882588268864227540007541F02258
:100A0D00C2AF75C820A8CCA9CDAA3A30CF010A75BE
:100A1D00C824D2AFAB3BAC3C883B893CC3E89BF8C8
:100A2D00E99C206908F9306602611C4176AD3D8A6A
:100A3D003DF9EA9DFA600478FF79FFAE3EAF3F8B3A
:100A4D003E8C3FA83BA93CC3E89EF8E99FF9C3E55E
:100A5D004113FBE54013FAE82AF540E93BF5415017
:100A6D00067540FF7541FF41C3AA40AB41AC40AD97
:100A7D00417E047F02C3EB9404400D1E1FC3EB9413
:100A8D00084005206A021E1FC3ED13FDEC13FCDEAA
:100A9D00F7C3EA9CFAEB9DFBEF6009C3E913F9E894
:100AAD0013F8DFF7EA28FAEB39FB8A408B41500641
:100ABD007BFF8B408B41C3EB94025002D2663069B1
:100ACD00047F0341EE7892E6FFC3E537948240112F
:100ADD000FC3E53794A040010FC3EF940640027F8A
:100AED00057E02E541C4540FF9E541C454F0F8E523
:100AFD0040C4540F28F8C3E89EFAE99400FB40095E
:100B0D00C3EA9402EB940050047A02E4FB6168AAF4
:100B1D0040AB41EBC4FEEAC4540F4EFCC3EA9CFA51
:100B2D00EB9400FBC3E813C313F8EA28FAEB340087
:100B3D00FB8A408B41C3EB94024002C2667802EB04
:100B4D00C4FE7B00EAC4540F4EFAC3EA98FA40057E
:100B5D00C3940250027A027892E6FF306002616817
:100B6D00855192855293D26043E680C3E49AF8E4AE
:100B7D009BF930660261F4E8FAE9FBD3E913FDE86D
:100B8D0013FC88518952C3EF94036038EF20E00DB8
:100B9D00E82CF8E93DF9ECFAEDFB020BBDE828F87D
:100BAD00E939F9C3E82402F8E93400F97AFE7BFF4C
:100BBD00C3EF9403400E8A538B54884D894E8C4F4E
:100BCD008D508128885389548A4D8B4E8C4F8D5072
:100BDD003069127553F07554FF754FF07550FF75F0
:100BED0051F07552FF8128E8FAD3E813FC8851C300
:100BFD00EF94036020EF20E007E82CF8ECFA811465
:100C0D00E8282402F87AFEC3EF940340088A53883B
:100C1D004D8C4F812888538A4D8C4FE568C33350D6
:100C2D0002646BF5683060028132753402D2604324
:100C3D00E680E52D54066034A840A941C3E913F9B7
:100C4D00E813F8C3E913F9E813F8306904E924400F
:100C5D00F9C2AF53E67F759100C3E498F594E4991A
:0F0C6D00F595759104D26043E680D2AF22D26430
:100C7C00754300752000306C03752040020C99D22E
:100C8C0064754300752040306C0375200078017941
:100C9C0001206620E52D54066002C2647914E541FA
:100CAC00C313700104F8C39414400278143069041F
:100CBC00781B791B206010E543600C306903D53438
:100CCC0004D26DA143913A0543E59B5440B52002F3
:100CDC00A12D30690908C3E89940011881C020642E
:100CEC000A08C3E8994002819981C0C264C2AF531B
:100CFC00E67F7591003066127594007595F87591C4
:100D0C0004D26043E680D2AF8199E5417EFFC333C4
:100D1C004005C3334001FEC3E49E759400F595A1D4
:100D2C000AC3E5339401500281993064028199D849
:100D3C0002A14181C0C26DC2AF53E67F759100859F
:100D4C005394855495759104854D92854E93D2603C
:100D5C0043E680D2AFE52D54066008206A020533C5
:100D6C00020D7F306D0D206C0A20640715811581F2
:100D7C0002161A2278003064027801E53775F00704
:100D8C00A4F9E5F028F5F0E9A2F013A2F113A2F210
:100D9C0013F537C394785003753778C3E537953816
:100DAC004008D265D297D295D293306002A1B68515
:100DBC004F92855093D26043E68022207D16C2AFBD
:100DCC00754202C294D296306202C293D2AF759F22
:100DDC0010020FB6C2AF754202C294D292306202B8
:100DEC00C297D2AF759F10020FB6307243207D2090
:100DFC00C2AF754203900134757B10D293C292300E
:100E0C006204C295C114D294D2AF759F13020FB66F
:100E1C00C2AF754203900134757B10D297C29630E5
:100E2C006204C295C134D294D2AF759F11020FB631
:100E3C00207D17C2AF75420390010FD2933062022E
:100E4C00C295D2AF759F13020FB6C2AF7542039015
:100E5C00010FD297306202C295D2AF759F11020F6B
:100E6C00B6207D16C2AF754204C296D29230620291
:100E7C00C295D2AF759F11020FB6C2AF754204C2B4
:100E8C0092D296306202C295D2AF759F13020FB602
:100E9C00307243207D20C2AF754205900123757BD3
:100EAC0040D295C294306204C297C1BAD296D2AFE6
:100EBC00759F10020FB6C2AF754205900145757B48
:100ECC0004D295C294306204C293C1DAD292D2AFEA
:100EDC00759F10020FB6207D17C2AF7542059001A9
:100EEC0005D295306202C297D2AF759F10020FB631
:100EFC00C2AF754205900119D2953062EBC293D204
:100F0C00AF759F10020FB6207D16C2AF754206C298
:100F1C0092D294306202C297D2AF759F13020FB671
:100F2C00C2AF754206C296D294306202C293D2AF5F
:100F3C00759F11020FB6307243207D20C2AF7542EF
:100F4C0001900145757B04D297C296306204C2931E
:100F5C00E160D292D2AF759F11020FB6C2AF75424B
:100F6C0001900123757B40D293C292306204C297E8
:100F7C00E180D296D2AF759F13020FB6207D17C2B7
:100F8C00AF754201900119D297306202C293D2AF71
:100F9C00759F11020FB6C2AF754201900105D29335
:100FAC00306202C297D2AF759F13C26522900103C3
:100FBC00757B00D297D295D293C296C294C292C23C
:100FCC00622278807607087607087601087604088E
:100FDC0076FF0876FF08760908760208760108760F
:100FEC0001788C76010876000876B40876FF0876CE
:100FFC00FF0876FF0876030876FF0876010876FF6F
:10100C000876250876D00876780876C8087604081D
:10101C0076FF08760108760008767A08760A087654
:10102C00010876010876000876FF0876002278879A
:10103C00E6FFC2727888C27DE630E102D27DC27EC4
:10104C007889E630E102D27EC3EF94026008758E97
:10105C0001D273021067758E00C273227880E61479
:0F106C009000809378A5F67881E6149000809329
:10107B0078A6F67886E61490008D9378A7F6789F7D
:10108B00E6F87005756B0001AEC3E8941140027869
:10109B0011E82828F56B256B256B28F56C256B283B
:1010AB0028F56D7886E6F539C3940250037539023D
:1010BB00789CE67538FFB402037538A0B40303754A
:1010CB00388278A3E61490009A93F566120FB92232
:1010DB00227896E6FA7897E6FB7888E6B40305C3A0
:1010EB00EB940EFB307F047A007BFFC3EB9AFCC3BF
:1010FB00948250027C827572000572EC8572F0A4AA
:10110B00C3E5F0947D40F222D27F11DC12054F1221
:10111B00054F7A007B007C10120545E55C2AFA74BA
:10112B00003BFBDCF37C04C3EB13FBEA13FADCF7A9
:10113B00FEC27F11DC22757C00757D00E5EF20E699
:10114B00037520000520903FFFE520146006901DDD
:10115B00FF1460009304600375EF1653D9BF7581BC
:10116B00C043FF8012054075EF0643B203E5B3247D
:10117B000220E70DF521E5E320E0068521B343E3EB
:10118B0001120FB97580FF75A40075F1B275D4DF2C
:10119B007590A975A5FC75F2FC75D50175A6017541
:1011AB00E241120FB9E4F8F6D8FD756801120FCEC3
:1011BB0012167178988673753001C2AF12055912E9
:1011CB00056912054F12057012054F1205771205AE
:1011DB004F121798120559120559120554C2AF75C3
:1011EB007C00757D0078FA79FA308507D9FBD8F742
:1011FB00021C00113A116811DB11DC78988673120E
:10120B000FB975881075890275C82475910475D846
:10121B004075A82275B80275E690759B80759D0088
:10122B0075D10E75BC5875BB0875BA1175E880126F
:10123B000540D2AF12089875360053DACF207E03E3
:10124B0043DA20307E0343DA1043DA01C2D8C2718D
:10125B00120559D2617B037A0CE55B70077A0CDBC4
:10126B00030211E812054F2070030211E8C270E56A
:10127B005CC3940240E1E52F541F855E5DF55EB5BE
:10128B005DD5DAD5C26153DACF207E0343DA203045
:10129B007E0343DA10C2D8C27178A2E67008D2740A
:1012AB00E52F54E0F52FC2757529001205543074E3
:1012BB0009C3E529940A4002D2751205457802301C
:1012CB0074027800C3E55C9840F0C2AF1205691256
:1012DB000569120569D2AF120559754C0012054507
:1012EB00788CE6C3940150030213D5E530C3940107
:1012FB0050030213D5757CA5757DF1207435C3E5BC
:10130B005C94FF50030213D5C2AF12057ED2AF120D
:10131B000554C3E55C940150EFC2AF120569120589
:10132B004A120569D2AF120554C3E55C94FF40E93C
:10133B0002181D7F05D27F11DC120554C2AFC27F8C
:10134B0011DCAE5CC3E55C947FD2AF500261E51259
:10135B000540C2AF12057ED2AFDFDA3113C3EE9474
:10136B00057897F61205591217A07F0AD27F11DC68
:10137B00120554C2AFC27F11DCAE5CC3E55C947F37
:10138B00D2AF50E6120540C2AF12056912054A12E0
:10139B000569D2AFDFD63113EE24037896F6F879D0
:1013AB0097E7C394824003985006E824827897F617
:1013BB001205591216B31217CF12055411DCC3E5DF
:1013CB005C94FF5002610002181D757C00757D0056
:1013DB00C3E55C954C4003855C4C12055478017950
:1013EB0088E7B403027805C3E55C98400241E8C284
:1013FB00AF12057E12057E12057ED2AF120559750E
:10140B003000E4F531F5320531E531F4703F05324A
:10141B00789AE67819146012783214600D787D147E
:10142B00600878FA146003753200C3E53298401DEA
:10143B00120FB9120540153275310078998673C2B7
:10144B00AF12057ED2AF7898867312055412054AF7
:10145B00E52A700530740221E878012074027806C1
:0D146B00C3E55C9840A1120554E52A70030A
:101478000211E8C2AF120FB9E4F522F523F524F5FD
:1014880025F526F567D2AF7885E6C333F565E4F52B
:1014980044F545F546F547F548F570F52CF52DF575
:1014A8003775700875BB1012054012092930EDFD1B
:1014B800A8BDA9BEE97001F8887112092D757008D8
:1014C80075BB10113AC2AF7561FF1209E68522613A
:1014D800852262852263D2AF7522017524017525A4
:1014E80001752601856069756A017888E6B4030785
:1014F800C27D307602D27DD268D269753300120F70
:1015080013120F42120A06120A0D120A06120A0DC7
:10151800120A06120C8B12065F120D80120DC712EA
:101528000A0D120C7A306E031206FF2066031208A9
:1015380052306603120882120D80120DF6120A0D3F
:10154800120C8B306E0312073B120D80120E6D12B7
:101558000A0D120C7A306E03120799120D80120EC2
:101568009C120A0D120C8B306E031207F6120D80B6
:10157800120F13120A0D120929120C7A120D801279
:101588000F4212092D120A0D30692C856461856499
:1015980062856069756A0179187A0CC3E5339940E8
:1015A80009C269D26A8A350215BFC3E55C94014055
:1015B8000302151B021622306A1D206C1AE5351429
:1015C8007006C26AD26BA11BF535C3E55C94014075
:1015D8000302151B021622753600C3E55F9401400D
:1015E80009856462856069756A0178FA79A4E7609B
:1015F800027803C3E55F985021307404E52A601A25
:1016080078F0306C058564617820C3E54198500214
:10161800A11B0536E55C6002C125753600C2AF1214
:101628000FB97887E6FE7602113A7887EEF6E4F588
:1016380022F523F524F525F526F565752C00752D7D
:1016480000D2AF120554120FB978A4E66006C2970B
:10165800C295C293307406E52A700221E8788DE6B7
:10166800C39401400241C5810D901A0D78201216CD
:10167800F5E520B4A50CA31216F5E520B45A03022B
:101688001693120FCE1216B30216B2901A03788070
:101698007B0A1216F5A308DBF9901A0F788C7B19D0
:1016A8001216F5A308DBF9901A2822C2AF121738D0
:1016B800121715901A00740E1216FAA37407121650
:1016C800FAA374151216FA901A0378807B0A121678
:1016D800F9A308DBF9901A0F788C7B191216F9A375
:1016E80008DBF912174B121729901A2822E493F6EF
:1016F80022E6438F01538FFDFFC3E583941C40010D
:1017080022EF857CB7857DB7F0538FFE22438F0289
:10171800438F01857CB7857DB7901A0DF0538FFCF8
:1017280022901A0D74A5D1FA901A0E745AD1FA2281
:101738007A3079D07820901A40D1F5E520F709A3BE
:10174800DAF7227A3079D0901A40E7D1FA09A3DA89
:10175800F922AB74A875BB01027980BB02027981BA
:10176800BB03027982BB04027994BB05027983BB6F
:1017780006027986BB07027992BB08027987BB0902
:1017880002799CBB0A027988BB0B027989E8F722A7
:101798007C05120559DCFB22C2AF120569120570DF
:1017A80012057712057E12054A1205691205701294
:1017B800057712057E12054A120569120570120591
:1017C8007712057ED2AF22C2AF12057E12057712BC
:1017D800057012056912054A12057E120577120571
:1017E8007012056912054A12057E120577120570F6
:1017F800120569D2AF22AE74AF75C2AF1205691275
:10180800056912056912054ADEF212057E12054ABB
:10181800DFF8D2AF221217A0121798121798757412
:10182800017575017576001217FE7C05AD5C120511
:1018380059C3ED955C70F5C3E55C9401400AC3E5B6
:101848005C94FF403702186112175A1216B3121728
:10185800A0C2AF75EF16121798DCD10576C3E576EE
:0E1868009403500280C11217980575E57414A0
:1018760090009F93F808C3E57598500280A8121748
:10188600981217980574C3E574940C50028094124C
:0D1896000FCE1216B3C2AF75EF16121798E1
:0319FD0002114193
:101A00000E071507070104FFFF09020101A55A018E
:101A100000B4FFFFFF03FF01FF25D078C804FF01DA
:091A200000FF0A010100FF00FFB4
:101A400023536B79494949333041232020202020FA
:101A500023424C48454C4923463333302320202031
:101A60002020202020202020202020202020202076
:101C0000C2AFC2D353D9BF7581C043B20343FF8073
:101C1000752438752503B1DC7529A5752AF175E29F
:101C20004043F12053A4DF75D4FFD2857DFA7803B9
:101C300079E67C10752200752300901DE97B0675FE
:101C400024987525013085028145208508D8FBD967
:101C5000F9DCF781B7308508D8FBD9F9DCF781B713
:101C6000B19CE493A3C39A6004DDC381B7DBDBB10D
:101C70008E6002812E7B08E493FAA3B16FDBF87AC1
:101C800030B16F752200752300B18EEAFCEBFDC305
:101C9000ED94FE400EB18E8A278B28ED30E0048A49
:101CA000828B83B18E7AC270D8C3ED94FE601950D6
:101CB000CEBD002BEC600F7520007521FF7529004B
:101CC000752A000200008100A827A9280809D80465
:101CD000D90281DCB192EA89AAF281CE0D81A3C337
:101CE000ED94035053EDA2E092007AC5C3E58294CF
:101CF00000E583941C508A200010438F02438F011B
:101D00008529B7852AB7F0300029A827A92808090E
:101D1000438F01538FFDD804D902A133C3E58394C7
:101D20001C4003A3A11689AAE28529B7852AB7F02A
:101D3000A3A116538FFC817F7AC1BD030CE493A34A
:101D4000FAB153DCF8B14B817F8181AA22AB23B178
:101D50006FEBFAEA6222752608C3E52313F523E543
:101D60002213F52250066323A0632201D526EAB18F
:101D7000DCB1DC75260AEAF4200102D285300102CA
:101D8000C285B1DCC3134002C201D526EB22B19259
:101D9000EAFB208502A192308502A197752608AE44
:101DA00024AF25C3EF13FFEE13FEB1E0B1DCC3EAAD
:101DB000133085024480FA30E703632201C3E52330
:101DC00013F523E52213F52250066323A0632201B5
:101DD000D526D9E52265236523F52222AE24AF2539
:101DE0000E0FDEFEDFFCD20122424C48656C6934E6
:071DF000373163F3300601F7
:00000001FF
